:10000000FFC0FEC0FDC0FCC0FBC0FAC0F9C0F8C014
:06001000F7C0F6C0F5C0C8
:10020000F89400E00BBF09BF00E808B904E101BDA4
:1002100004E001BD0FED0DBF00E007BB06E301BB2D
:1002200000E702BB00B308700030D1F300E302BB6B
:1002300000E007BB06B30093B00016B31017B1F788
:100240002FD100E002BB06E701BB00E002BB0CD0EF
:100250008FD08330E9F7F89450D0C8F359D010F418
:100260006FD0A8F3B8D0F3CF03E009B908E10AB919
:1002700006E701BB00E002BB1CB10CB19927B0E05E
:10028000A0E699273327882708950CB970270BB16A
:1002900000720030E1F30895F0E0E0E626E002E0CD
:1002A000F4DF01912A95203019F0EFDF3196F9CF74
:1002B00003E0EBDF072FE9DF089537D104E0032BDC
:1002C00002BB05E1E2DF00E0E0DF00E002BB0895F1
:1002D0002CD12091B400203039F404E0032B02BB70
:1002E00006E0D3DF00E0D1DF00E002BB089504E0C8
:1002F000032B02BB012FC9DF0895F0E0E0E6E90F10
:100300000081071719F0D9DF08940895889408959B
:1003100022272093B400F0E0E0E601912091B100A3
:10032000021761F401912091B200021739F4019192
:100330002091B300021711F4889408950894089549
:1003400022272093B400F0E0E0E6019120E30217B9
:1003500069F4019120E3021749F4019120E30217A7
:1003600029F421E02093B400889408950894089516
:100370001BB1107809F408951871103029F51CB1DB
:100380001F3F19F18030A1F0823059F01D93712781
:10039000133019F4000082E012C093959233A8F450
:1003A0000EC01D93939510E01D9383E0F89407C051
:1003B000123029F49927B0E0A0E672E081E01BB189
:1003C0001871103011F408951CB100009927B0E0A5
:1003D000A0E688270895F0E0E0E60381073549F0BC
:1003E0000235D9F0023731F1053469F0043559F09E
:1003F00008956EDF3396D0E0C2E92DE077D02EE08D
:1004000030E225D0089564DF3396D0E0C2E92FE1D1
:100410006DD02FE130E21BD008953396D0E0C2E9D1
:1004200024E064D024E030E112D02AE025D02AE094
:1004300063D008953396D0E0C2E924E057D024E099
:1004400030E105D023E118D023E156D00895F0E043
:10045000E2E90FEF07BB32BB00B308700030E1F3F5
:10046000019108BB00B308700030E1F72A952030F5
:1004700099F700E007BB0895F0E0E0E600E007BB75
:1004800000B308700030E1F306B3019300B30870C5
:100490000030E1F72A95203099F700E007BB089576
:1004A0004091B00050E35093B1005093B20050938C
:1004B000B300042F8894044630F0402F61E0560FBB
:1004C0005093B100F6CF50E0042F88940A4040F0DA
:1004D000402F5091B20061E0560F5093B200F4CF1C
:1004E0005091B300540F5093B300089501910993B4
:1004F0002A952223D9F7089518D0F0E0E0E604E029
:1005000002BB02E07727C1DE0191BFDE2A952223DC
:1005100009F0FACF03E0B9DE072FB7DE00E0B5DE61
:10052000332732BB032F02BB089545E00FEF0A9536
:100530000030E9F74A954030C9F708954E65747761
:100540006F726B20436F6E74726F6C2050726F63AA
:100550006573736F72212B3132333435363738215E
:00000001FF
